:10503C0033302E322020200006012C034D056E0744
:10504C008F09A70B0000000000000032006400C8AC
:10505C00012C015E019001C201FC022E026102943E
:10506C0002C702FA032C035F039203C503F8042A58
:10507C00045D049004C304F60528055B058E05C188
:10508C0005F406260659068C06BF06F207240757B8
:10509C00078A07BD07F008220855088808BB08EEE8
:1050AC0009210953098609B909EC0A1F0A510A8416
:1050BC000AB70AEA0B1D0B4F0B820BB50BE80C1B46
:1050CC000C4D0C800CB30CE60D190D4B0D7E0DB177
:1050DC000DE40E170E490E7C0EAF0EE20F150F47A6
:1050EC000F7A0FAD0FE010131045107810AB10DED7
:1050FC0011111144117611A911DC120F1242127404
:10510C0012A712DA130D1340137213A513D8140B34
:10511C00143E147014A314D61509153C156E15A164
:10512C0015D41607163A166C169F16D21705173893
:10513C00176A179D17D0180318361868189B18CEC5
:10514C00190119341967199919CC19FF1A321A65F2
:10515C001A971ACA1AFD1B301B631B951BC81BFB25
:10516C001C2E1C611C931CC61CF91D2C1D5F1D9153
:10517C001DC41DF71E2A1E5D1E8F1EC21EF51F2884
:10518C001F5B1F8D1FC01FF320262059208B20BEB4
:10519C0020F121242157218921BC21EF22222255E3
:1051AC00228822BA22ED23202353238623B823EB13
:1051BC00241E2451248424B624E9251C254F258241
:1051CC0025B425E7261A264D268026B226E5271873
:1051DC00274B277E27B027E328162849287C28AEA2
:1051EC0028E129142947297A29AC29DF2A122A45D2
:1051FC002A782AAB2ADD2B102B432B762BA92BDB01
:10520C002C0E2C412C742CA72CD92D0C2D3F2D722F
:10521C002DA52DD72E0A2E3D2E702EA32ED52F0860
:10522C002F3B2F6E2FA12FD330063039306C309F8F
:10523C0030D131043137316A319D31CF32023235C0
:10524C003268329B32CE330033333366339933CCEE
:10525C0033FE34313464349734CA34FC352F356220
:10526C00359535C835FA362D3660369336C636F850
:10527C00372B375E379137C437F63829385C388F7F
:10528C0038C238F43927395A398D39C039F23A25B0
:10529C003A583A8B3ABE3AF03B233B563B893BBCDF
:1052AC003BEF3C213C543C873CBA3CED3D1F3D520E
:1052BC003D853DB83DEB3E1D3E503E833EB63EE93E
:1052CC003F1B3F4E3F813FB43FE74019404C407F6E
:1052DC0040B240E54117414A417D41B041E342159E
:1052EC004248427B42AE42E143134346437943ACCE
:1052FC0043DF44124444447744AA44DD45104542FC
:10530C00457545A845DB460E4640467346A646D92C
:10531C00470C473E477147A447D7480A483C486F5B
:10532C0048A248D54908493A496D49A049D34A068B
:10533C004A384A6B4A9E4AD14B044B364B694B9CBC
:10534C004BCF4C024C354C674C9A4CCD4D004D33E9
:10535C004D654D984DCB4DFE4E314E634E964EC91C
:10536C004EFC4F2F4F614F944FC74FFA502D505F4B
:10537C00509250C550F8512B515D519051C351F67C
:10538C005229525B528E52C152F453275359538CAB
:10539C0053BF53F254255457548A54BD54F05523DB
:1053AC005556558855BB55EE56215654568656B90A
:1053BC0056EC571F5752578457B757EA581D585039
:1053CC00588258B558E8591B594E598059B359E66B
:1053DC005A195A4C5A7E5AB15AE45B175B4A5B7C99
:1053EC005BAF5BE25C155C485C7A5CAD5CE05D13CA
:1053FC005D465D795DAB5DDE5E115E445E775EA9F8
:10540C005EDC5F0F5F425F755FA75FDA600D604027
:10541C00607360A560D8610B613E617161A361D658
:10542C006209623C626F62A162D46307633A636D86
:10543C00639F63D264056438646B649D64D06503B8
:10544C0065366569659B65A765B265BD65C865D33D
:10545C0065DE65E965F465FF660A66156620662BF0
:10546C0066366641664C66576662666D667866831C
:10547C00668E669966A466AF66BA66C566D066DB4C
:10548C0066E666F166FC67086713671E6729673472
:10549C00673F674A67556760676B67766781678C9C
:1054AC00679767A267AD67B867C367CE67D967E4CC
:1054BC0067EF67FA68056810681B68266831683CF6
:1054CC0068476852685D68686874687F688A689520
:1054DC0068A068AB68B668C168CC68D768E268ED4C
:1054EC0068F86903690E69196924692F693A694575
:1054FC006950695B69666971697C69876992699DA4
:10550C0069A869B369BE69C969D569E069EB69F6CF
:10551C006A016A0C6A176A226A2D6A386A436A4EF3
:10552C006A596A646A6F6A7A6A856A906A9B6AA623
:10553C006AB16ABC6AC76AD26ADD6AE86AF36AFE53
:10554C006B096B146B1F6B2A6B356B416B4C6B5778
:10555C006B626B6D6B786B836B8E6B996BA46BAFA3
:10556C006BBA6BC56BD06BDB6BE66BF16BFC6C07D2
:10557C006C126C1D6C286C336C3E6C496C546C5FFB
:10558C006C6A6C756C806C8B6C966CA26CAD6CB828
:10559C006CC36CCE6CD96CE46CEF6CFA6D056D1051
:1055AC006D1B6D266D316D3C6D476D526D5D6D687B
:1055BC006D736D7E6D896D946D9F6DAA6DB56DC0AB
:1055CC006DCB6DD66DE16DEC6DF76E026E0E6E19D6
:1055DC006E246E2F6E3A6E456E506E5B6E666E71FB
:1055EC006E7C6E876E926E9D6EA86EB36EBE6EC92B
:1055FC006ED46EDF6EEA6EF56F006F0B6F166F2157
:10560C006F2C6F376F426F4D6F586F636F6E6F7A81
:10561C006F856F906F9B6FA66FB16FBC6FC76FD2AA
:10562C006FDD6FE86FF36FFE70097014701F702AD6
:10563C0070357040704B70567061706C7077708202
:10564C00708D709870A370AE70B970C470CF70DB31
:10565C0070E670F170FC71077112711D7128713355
:10566C00713E71497154715F716A71757180718B82
:10567C00719671A171AC71B771C271CD71D871E3B2
:10568C0071EE71F97204720F721A72257230723BDC
:10569C0072477252725D72687273727E7289729402
:1056AC00729F72AA72B572C072CB72D672E172EC32
:1056BC0072F77302730D73187323732E733973445B
:1056CC00734F735A73657370737B73867391739C8A
:1056DC0073A873B373BE73C973D473DF73EA73F5B2
:1056EC007400740B74167421742C74377442744DDA
:1056FC0074587463746E74797484748F749A74A50A
:10570C0074B074BB74C674D174DC74E774F274FD39
:10571C0075087514751F752A75357540754B75565A
:10572C007561756C75777582758D759875A375AE89
:10573C0075B975C475CF75DA75E575F075FB7606B8
:10574C007611761C76277632763D76487653765EE1
:10575C00766976757680768B769676A176AC76B70A
:10576C0076C276CD76D876E376EE76F97704770F37
:10577C00771A77257730773B77467751775C776761
:10578C007772777D77887793779E77A977B477BF91
:10579C0077CA77D577E177EC77F77802780D7818B8
:1057AC007823782E78397844784F785A78657870E1
:1057BC00787B78867891789C78A778B278BD78C811
:1057CC0078D378DE78E978F478FF790A791579203E
:1057DC00792B79367941794D79587963796E797964
:1057EC007984798F799A79A579B079BB79C679D191
:1057FC0079DC79E779F279FD7A087A137A1E7A29BD
:10580C007A347A3F7A4A7A557A607A6B7A767A81E8
:10581C007A8C7A977AA27AAE7AB97AC47ACF7ADA13
:10582C007AE57AF07AFB7B067B117B1C7B277B323B
:10583C007B3D7B487B537B5E7B697B747B7F7B8A68
:10584C007B957BA07BAB7BB67BC17BCC7BD77BE298
:10585C007BED7BF87C037C0E7C1A7C257C307C3BBE
:10586C007C467C517C5C7C677C727C7D7C887C93E8
:10587C007C9E7CA97CB47CBF7CCA7CD57CE07CEB18
:10588C007CF67D017D0C7D177D227D2D7D387D4341
:10589C007D4E7D597D647D6F7D7B7D867D917D9C6C
:1058AC007DA77DB27DBD7DC87DD37DDE7DE97DF498
:1058BC007DFF7E0A7E157E207E2B7E367E417E4CC1
:1058CC007E577E627E6D7E787E837E8E7E997EA4F0
:1058DC007EAF7EBA7EC57ED07EDB7EE77EF27EFD1D
:1058EC007F087F137F1E7F297F347F3F7F4A7F5540
:1058FC007F607F6B7F767F817F8C7F977FA27FAD70
:10590C007FB87FC37FCE7FD97FE47FEF7FFA80059E
:10591C008010801B80268031803C80488053805EC4
:10592C0080698074807F808A809580A080AB80B6EF
:10593C0080C180CC80D780E280ED80F88103810E1D
:10594C0081198124812F813A81458150815B816647
:10595C008171817C81878192819D81A881B481BF75
:10596C0081CA81D581E081EB81F68201820C82179C
:10597C008222822D82388243824E82598264826FC7
:10598C00827A82858290829B82A682B182BC82C7F7
:10599C0082D282DD82E882F382FE83098314832023
:1059AC00832B83368341834C83578362836D837847
:1059BC008383838E839983A483AF83BA83C583D077
:1059CC0083DB83E683F183FC84078412841D8428A3
:1059DC008433843E84498454845F846A84758481CE
:1059EC00848C849784A284AD84B884C384CE84D9F7
:1059FC0084E484EF84FA85058510851B8526853122
:105A0C00853C85478552855D85688573857E85894E
:105A1C008594859F85AA85B585C085CB85D685E17E
:105A2C0085ED85F88603860E86198624862F863AA0
:105A3C0086458650865B86668671867C86878692CE
:105A4C00869D86A886B386BE86C986D486DF86EAFE
:105A5C0086F58700870B87168721872C8737874227
:105A6C00874E87598764876F877A87858790879B4E
:105A7C0087A687B187BC87C787D287DD87E887F37E
:105A8C0087FE88098814881F882A88358840884BA7
:105A9C0088568861886C88778882888D889888A3D6
:105AAC0088AE88BA88C588D088DB88E688F188FCFF
:105ABC0089078912891D89288933893E8949895426
:105ACC00895F896A89758980898B899689A189AC56
:105ADC0089B789C289CD89D889E389EE89F98A0485
:105AEC008A0F8A1B8A268A318A3C8A478A528A5DA7
:105AFC008A688A738A7E8A898A948A9F8AAA8AB5D6
:105B0C008AC08ACB8AD68AE18AEC8AF78B028B0D03
:105B1C008B188B238B2E8B398B448B4F8B5A8B652D
:105B2C008B708B7B8B878B928B9D8BA88BB38BBE57
:105B3C008BC98BD48BDF8BEA8BF58C008C0B8C1682
:105B4C008C218C2C8C378C428C4D8C588C638C6EAD
:105B5C008C798C848C8F8C9A8CA58CB08CBB8CC6DD
:105B6C008CD18CDC8CE78CF38CFE8D098D148D1F05
:105B7C008D2A8D358D408D4B8D568D618D6C8D772D
:105B8C008D828D8D8D988DA38DAE8DB98DC48DCF5D
:105B9C008DDA8DE58DF08DFB8E068E118E1C8E2789
:105BAC008E328E3D8E488E548E5F8E6A8E758E80B0
:105BBC008E8B8E968EA18EAC8EB78EC28ECD8ED8DD
:105BCC008EE38EEE8EF98F048F0F8F1A8F258F3008
:105BDC008F3B8F468F518F5C8F678F728F7D8F8835
:105BEC008F938F9E8FA98FB48FC08FCB8FD68FE161
:105BFC008FEC8FF79002900D90189023902E903987
:105C0C009044904F905A90659070907B90869091B4
:105C1C00909C90A790B290BD90C890D390DE90E9E4
:105C2C0090F490FF910A91159121912C913791420A
:105C3C00914D91589163916E91799184918F919A34
:105C4C0091A591B091BB91C691D191DC91E791F264
:105C5C0091FD92089213921E92299234923F924A8D
:105C6C0092559260926B92769281928D929892A3B9
:105C7C0092AE92B992C492CF92DA92E592F092FBE4
:105C8C0093069311931C93279332933D934893530C
:105C9C00935E93699374937F938A939593A093AB3C
:105CAC0093B693C193CC93D793E293EE93F9940468
:105CBC00940F941A94259430943B94469451945C8C
:105CCC0094679472947D94889493949E94A994B4BC
:105CDC0094BF94CA94D594E094EB94F69501950CEA
:105CEC0095179522952D95389543954E955A956512
:105CFC009570957B95869591959C95A795B295BD3C
:105D0C0095C895D395DE95E995F495FF960A961569
:105D1C009620962B96369641964C96579662966D93
:105D2C0096789683968E969996A496AF96BA96C6C2
:105D3C0096D196DC96E796F296FD97089713971EE8
:105D4C0097299734973F974A97559760976B977613
:105D5C009781978C979797A297AD97B897C397CE43
:105D6C0097D997E497EF97FA98059810981B98276E
:105D7C009832983D98489853985E98699874987F93
:105D8C00988A989598A098AB98B698C198CC98D7C3
:105D9C0098E298ED98F89903990E99199924992FEE
:105DAC00993A99459950995B99669971997C99871B
:105DBC009993999E99A999B499BF99CA99D599E043
:105DCC0099EB99F69A019A0C9A179A229A2D9A386D
:105DDC009A439A4E9A599A649A6F9A7A9A859A909B
:105DEC009A9B9AA69AB19ABC9AC79AD29ADD9AE8CB
:105DFC009AF49AFF9B0A9B159B209B2B9B369B41ED
:105E0C009B4C9B579B629B6D9B789B839B8E9B991A
:105E1C009BA49BAF9BBA9BC59BD09BDB9BE69BF14A
:105E2C009BFC9C079C129C1D9C289C339C3E9C4973
:105E3C009C549C609C6B9C769C819C8C9C979CA29B
:105E4C009CAD9CB89CC39CCE9CD99CE49CEF9CFACA
:105E5C009D059D109D1B9D269D319D3C9D479D52F2
:105E6C009D5D9D689D739D7E9D899D949D9F9DAA22
:105E7C009DB59DC19DCC9DD79DE29DED9DF89E034A
:105E8C009E0E9E199E249E2F9E3A9E459E509E5B72
:105E9C009E669E719E7C9E879E929E9D9EA89EB3A2
:105EAC009EBE9EC99ED49EDF9EEA9EF59F009F0BD0
:105EBC009F169F219F2D9F389F439F4E9F599F64F4
:105ECC009F6F9F7A9F859F909F9B9FA69FB19FBC22
:105EDC009FC79FD29FDD9FE89FF39FFEA009A01450
:105EEC00A01FA02AA035A040A04BA056A061A06C7A
:105EFC00A077A082A08DA099A0A4A0AFA0BAA0C5A5
:105F0C00A0D0A0DBA0E6A0F1A0FCA107A112A11DCE
:105F1C00A128A133A13EA149A154A15FA16AA175F9
:105F2C00A180A18BA196A1A1A1ACA1B7A1C2A1CD29
:105F3C00A1D8A1E3A1EEA1FAA205A210A21BA22650
:105F4C00A231A23CA247A252A25DA268A273A27E79
:105F5C00A289A294A29FA2AAA2B5A2C0A2CBA2D6A9
:105F6C00A2E1A2ECA2F7A302A30DA318A323A32ED4
:105F7C00A339A344A34FA35AA366A371A37CA387FD
:105F8C00A392A39DA3A8A3B3A3BEA3C9A3D4A3DF29
:105F9C00A3EAA3F5A400A40BA416A421A42CA43753
:105FAC00A442A44DA458A463A46EA479A484A48F81
:105FBC00A49AA4A5A4B0A4BBA4C7A4D2A4DDA4E8AD
:105FCC00A4F3A4FEA509A514A51FA52AA535A540D3
:105FDC00A54BA556A561A56CA577A582A58DA59801
:105FEC00A5A3A5AEA5B9A5C4A5CFA5DAA5E5A5F031
:105FFC00A5FBA606A611A61CA627A633A63EA64957
:10600C00A654A65FA66AA675A680A68BA696A6A180
:10601C00A6ACA6B7A6C2A6CDA6D8A6E3A6EEA6F9B0
:10602C00A704A70FA71AA725A730A73BA746A751D8
:10603C00A75CA767A772A77DA788A794A79FA7AA05
:10604C00A7B5A7C0A7CBA7D6A7E1A7ECA7F7A8022F
:10605C00A80DA818A823A82EA839A844A84FA85A58
:10606C00A865A870A87BA886A891A89CA8A7A8B288
:10607C00A8BDA8C8A8D3A8DEA8E9A8F4A900A90BB4
:10608C00A916A921A92CA937A942A94DA958A963D8
:10609C00A96EA979A984A98FA99AA9A5A9B0A9BB08
:1060AC00A9C6A9D1A9DCA9E7A9F2A9FDAA08AA1336
:1060BC00AA1EAA29AA34AA3FAA4AAA55AA60AA6C5F
:1060CC00AA77AA82AA8DAA98AAA3AAAEAAB9AAC488
:1060DC00AACFAADAAAE5AAF0AAFBAB06AB11AB1CB5
:1060EC00AB27AB32AB3DAB48AB53AB5EAB69AB74E0
:1060FC00AB7FAB8AAB95ABA0ABABABB6ABC1ABCD0F
:10610C00ABD8ABE3ABEEABF9AC04AC0FAC1AAC2533
:10611C00AC30AC3BAC46AC51AC5CAC67AC72AC7D5F
:10612C00AC88AC93AC9EACA9ACB4ACBFACCAACD58F
:10613C00ACE0ACEBACF6AD01AD0CAD17AD22AD2DBA
:10614C00AD39AD44AD4FAD5AAD65AD70AD7BAD86DF
:10615C00AD91AD9CADA7ADB2ADBDADC8ADD3ADDE0F
:10616C00ADE9ADF4ADFFAE0AAE15AE20AE2BAE363A
:10617C00AE41AE4CAE57AE62AE6DAE78AE83AE8E67
:10618C00AE9AAEA5AEB0AEBBAEC6AED1AEDCAEE78F
:10619C00AEF2AEFDAF08AF13AF1EAF29AF34AF3FB9
:1061AC00AF4AAF55AF60AF6BAF76AF81AF8CAF97E7
:1061BC00AFA2AFADAFB8AFC3AFCEAFD9AFE4AFEF17
:1061CC00AFFAB006B011B01CB027B032B03DB04839
:1061DC00B053B05EB069B074B07FB08AB095B0A067
:1061EC00B0ABB0B6B0C1B0CCB0D7B0E2B0EDB0F897
:1061FC00B103B10EB119B124B12FB13AB145B150BF
:10620C00B15BB167B172B17DB188B193B19EB1A9E7
:10621C00B1B4B1BFB1CAB1D5B1E0B1EBB1F6B20115
:10622C00B20CB217B222B22DB238B243B24EB2593E
:10623C00B264B26FB27AB285B290B29BB2A6B2B16E
:10624C00B2BCB2C7B2D3B2DEB2E9B2F4B2FFB30A97
:10625C00B315B320B32BB336B341B34CB357B362BE
:10626C00B36DB378B383B38EB399B3A4B3AFB3BAEE
:10627C00B3C5B3D0B3DBB3E6B3F1B3FCB407B4121C
:10628C00B41DB428B433B43FB44AB455B460B46B41
:10629C00B476B481B48CB497B4A2B4ADB4B8B4C36E
:1062AC00B4CEB4D9B4E4B4EFB4FAB505B510B51B9B
:1062BC00B526B531B53CB547B552B55DB568B573C6
:1062CC00B57EB589B594B5A0B5ABB5B6B5C1B5CCF1
:1062DC00B5D7B5E2B5EDB5F8B603B60EB619B6241A
:1062EC00B62FB63AB645B650B65BB666B671B67C46
:1062FC00B687B692B69DB6A8B6B3B6BEB6C9B6D476
:10630C00B6DFB6EAB6F5B700B70CB717B722B72D9C
:10631C00B738B743B74EB759B764B76FB77AB785C5
:10632C00B790B79BB7A6B7B1B7BCB7C7B7D2B7DDF5
:10633C00B7E8B7F3B7FEB809B814B81FB82AB83520
:10634C00B840B84BB856B861B86DB878B883B88E49
:10635C00B899B8A4B8AFB8BAB8C5B8D0B8DBB8E675
:10636C00B8F1B8FCB907B912B91DB928B933B93E9F
:10637C00B949B954B95FB96AB975B980B98BB996CD
:10638C00B9A1B9ACB9B7B9C2B9CDB9D9B9E4B9EFFA
:10639C00B9FABA05BA10BA1BBA26BA31BA3CBA471E
:1063AC00BA52BA5DBA68BA73BA7EBA89BA94BA9F4D
:1063BC00BAAABAB5BAC0BACBBAD6BAE1BAECBAF77D
:1063CC00BB02BB0DBB18BB23BB2EBB3ABB45BB50A2
:1063DC00BB5BBB66BB71BB7CBB87BB92BB9DBBA8CD
:1063EC00BBB3BBBEBBC9BBD4BBDFBBEABBF5BC00FC
:1063FC00BC0BBC16BC21BC2CBC37BC42BC4DBC5825
:10640C00BC63BC6EBC79BC84BC8FBC9ABCA6BCB152
:10641C00BCBCBCC7BCD2BCDDBCE8BCF3BCFEBD097B
:10642C00BD14BD1FBD2ABD35BD40BD4BBD56BD61A4
:10643C00BD6CBD77BD82BD8DBD98BDA3BDAEBDB9D4
:10644C00BDC4BDCFBDDABDE5BDF0BDFBBE06BE1201
:10645C00BE1DBE28BE33BE3EBE49BE54BE5FBE6A24
:10646C00BE75BE80BE8BBE96BEA1BEACBEB7BEC254
:10647C00BECDBED8BEE3BEEEBEF9BF04BF0FBF1A81
:10648C00BF25BF30BF3BBF46BF51BF5CBF67BF73AB
:10649C00BF7EBF89BF94BF9FBFAABFB5BFC0BFCBD4
:1064AC00BFD6BFE1BFECBFF7C002C00DC018C02300
:1064BC00C02EC039C044C04FC05AC065C070C07B2C
:1064CC00C086C091C09CC0A7C0B2C0BDC0C8C0D35C
:1064DC00C0DFC0EAC0F5C100C10BC116C121C12C7F
:1064EC00C137C142C14DC158C163C16EC179C184AC
:1064FC00C18FC19AC1A5C1B0C1BBC1C6C1D1C1DCDC
:10650C00C1E7C1F2C1FDC208C213C21EC229C23406
:10651C00C240C24BC256C261C26CC277C282C28D2B
:10652C00C298C2A3C2AEC2B9C2C4C2CFC2DAC2E55B
:10653C00C2F0C2FBC306C311C31CC327C332C33D85
:10654C00C348C353C35EC369C374C37FC38AC395B3
:10655C00C3A0C3ACC3B7C3C2C3CDC3D8C3E3C3EEDC
:10656C00C3F9C404C40FC41AC425C430C43BC44604
:10657C00C451C45CC467C472C47DC488C493C49E33
:10658C00C4A9C4B4C4BFC4CAC4D5C4E0C4EBC4F663
:10659C00C501C50DC518C523C52EC539C544C54F84
:1065AC00C55AC565C570C57BC586C591C59CC5A7B3
:1065BC00C5B2C5BDC5C8C5D3C5DEC5E9C5F4C5FFE3
:1065CC00C60AC615C620C62BC636C641C64CC6570B
:1065DC00C662C66DC679C684C68FC69AC6A5C6B035
:1065EC00C6BBC6C6C6D1C6DCC6E7C6F2C6FDC70862
:1065FC00C713C71EC729C734C73FC74AC755C7608B
:10660C00C76BC776C781C78CC797C7A2C7ADC7B8BA
:10661C00C7C3C7CEC7D9C7E5C7F0C7FBC806C811E3
:10662C00C81CC827C832C83DC848C853C85EC8690A
:10663C00C874C87FC88AC895C8A0C8ABC8B6C8C13A
:10664C00C8CCC8D7C8E2C8EDC8F8C903C90EC91967
:10665C00C924C92FC93AC946C951C95CC967C9728D
:10666C00C97DC988C993C99EC9A9C9B4C9BFC9CABA
:10667C00C9D5C9E0C9EBC9F6CA01CA0CCA17CA22E6
:10668C00CA2DCA38CA43CA4ECA59CA64CA6FCA7A12
:10669C00CA85CA90CA9BCAA6CAB2CABDCAC8CAD33E
:1066AC00CADECAE9CAF4CAFFCB0ACB15CB20CB2B66
:1066BC00CB36CB41CB4CCB57CB62CB6DCB78CB8392
:1066CC00CB8ECB99CBA4CBAFCBBACBC5CBD0CBDBC2
:1066DC00CBE6CBF1CBFCCC07CC13CC1ECC29CC34E9
:1066EC00CC3FCC4ACC55CC60CC6BCC76CC81CC8C12
:1066FC00CC97CCA2CCADCCB8CCC3CCCECCD9CCE442
:10670C00CCEFCCFACD05CD10CD1BCD26CD31CD3C6B
:10671C00CD47CD52CD5DCD68CD73CD7FCD8ACD9596
:10672C00CDA0CDABCDB6CDC1CDCCCDD7CDE2CDEDC1
:10673C00CDF8CE03CE0ECE19CE24CE2FCE3ACE45EA
:10674C00CE50CE5BCE66CE71CE7CCE87CE92CE9D19
:10675C00CEA8CEB3CEBECEC9CED4CEE0CEEBCEF646
:10676C00CF01CF0CCF17CF22CF2DCF38CF43CF4E69
:10677C00CF59CF64CF6FCF7ACF85CF90CF9BCFA699
:10678C00CFB1CFBCCFC7CFD2CFDDCFE8CFF3CFFEC9
:10679C00D009D014D01FD02AD035D040D04CD057EF
:1067AC00D062D06DD078D083D08ED099D0A4D0AF19
:1067BC00D0BAD0C5D0D0D0DBD0E6D0F1D0FCD10748
:1067CC00D112D11DD128D133D13ED149D154D15F71
:1067DC00D16AD175D180D18BD196D1A1D1ACD1B8A0
:1067EC00D1C3D1CED1D9D1E4D1EFD1FAD205D210C7
:1067FC00D21BD226D231D23CD247D252D25DD268F1
:10680C00D273D27ED289D294D29FD2AAD2B5D2C020
:10681C00D2CBD2D6D2E1D2ECD2F7D302D30DD3194C
:10682C00D324D32FD33AD345D350D35BD366D37170
:10683C00D37CD387D392D39DD3A8D3B3D3BED3C9A0
:10684C00D3D4D3DFD3EAD3F5D400D40BD416D421CC
:10685C00D42CD437D442D44DD458D463D46ED479F8
:10686C00D485D490D49BD4A6D4B1D4BCD4C7D4D220
:10687C00D4DDD4E8D4F3D4FED509D514D51FD52A4C
:10688C00D535D540D54BD556D561D56CD577D58278
:10689C00D58DD598D5A3D5AED5B9D5C4D5CFD5DAA8
:1068AC00D5E6D5F1D5FCD607D612D61DD628D633CB
:1068BC00D63ED649D654D65FD66AD675D680D68BF8
:1068CC00D696D6A1D6ACD6B7D6C2D6CDD6D8D6E328
:1068DC00D6EED6F9D704D70FD71AD725D730D73B52
:1068EC00D746D752D75DD768D773D77ED789D79479
:1068FC00D79FD7AAD7B5D7C0D7CBD7D6D7E1D7ECA8
:10690C00D7F7D802D80DD818D823D82ED839D844D0
:10691C00D84FD85AD865D870D87BD886D891D89CFF
:10692C00D8A7D8B3D8BED8C9D8D4D8DFD8EAD8F528
:10693C00D900D90BD916D921D92CD937D942D94D4F
:10694C00D958D963D96ED979D984D98FD99AD9A57F
:10695C00D9B0D9BBD9C6D9D1D9DCD9E7D9F2D9FDAF
:10696C00DA08DA13DA1FDA2ADA35DA40DA4BDA56D1
:10697C00DA61DA6CDA77DA82DA8DDA98DAA3DAAEFF
:10698C00DAB9DAC4DACFDADADAE5DAF0DAFBDB062E
:10699C00DB11DB1CDB27DB32DB3DDB48DB53DB5E57
:1069AC00DB69DB74DB7FDB8BDB96DBA1DBACDBB782
:1069BC00DBC2DBCDDBD8DBE3DBEEDBF9DC04DC0FAD
:1069CC00DC1ADC25DC30DC3BDC46DC51DC5CDC67D7
:1069DC00DC72DC7DDC88DC93DC9EDCA9DCB4DCBF07
:1069EC00DCCADCD5DCE0DCECDCF7DD02DD0DDD182F
:1069FC00DD23DD2EDD39DD44DD4FDD5ADD65DD7057
:106A0C00DD7BDD86DD91DD9CDDA7DDB2DDBDDDC886
:106A1C00DDD3DDDEDDE9DDF4DDFFDE0ADE15DE20B3
:106A2C00DE2BDE36DE41DE4CDE58DE63DE6EDE79DA
:106A3C00DE84DE8FDE9ADEA5DEB0DEBBDEC6DED106
:106A4C00DEDCDEE7DEF2DEFDDF08DF13DF1EDF2932
:106A5C00DF34DF3FDF4ADF55DF60DF6BDF76DF815E
:106A6C00DF8CDF97DFA2DFADDFB9DFC4DFCFDFDA8A
:106A7C00DFE5DFF0DFFBE006E011E01CE027E032B1
:106A8C00E03DE048E053E05EE069E074E07FE08ADE
:106A9C00E095E0A0E0ABE0B6E0C1E0CCE0D7E0E20E
:106AAC00E0EDE0F8E103E10EE119E125E130E13B35
:106ABC00E146E151E15CE167E172E17DE188E1935E
:106ACC00E19EE1A9E1B4E1BFE1CAE1D5E1E0E1EB8E
:106ADC00E1F6E201E20CE217E222E22DE238E243B7
:106AEC00E24EE259E264E26FE27AE286E291E29CE3
:106AFC00E2A7E2B2E2BDE2C8E2D3E2DEE2E9E2F40E
:106B0C00E2FFE30AE315E320E32BE336E341E34C36
:106B1C00E357E362E36DE378E383E38EE399E3A465
:106B2C00E3AFE3BAE3C5E3D0E3DBE3E6E3F2E3FD93
:106B3C00E408E413E41EE429E434E43FE44AE455B5
:106B4C00E460E46BE476E481E48CE497E4A2E4ADE5
:106B5C00E4B8E4C3E4CEE4D9E4E4E4EFE4FAE50514
:106B6C00E510E51BE526E531E53CE547E552E55E3C
:106B7C00E569E574E57FE58AE595E5A0E5ABE5B665
:106B8C00E5C1E5CCE5D7E5E2E5EDE5F8E603E60E93
:106B9C00E619E624E62FE63AE645E650E65BE666BD
:106BAC00E671E67CE687E692E69DE6A8E6B3E6BFEC
:106BBC00E6CAE6D5E6E0E6EBE6F6E701E70CE71712
:106BCC00E722E72DE738E743E74EE759E764E76F3D
:106BDC00E77AE785E790E79BE7A6E7B1E7BCE7C76D
:106BEC00E7D2E7DDE7E8E7F3E7FEE809E814E81F9A
:106BFC00E82BE836E841E84CE857E862E86DE878BD
:106C0C00E883E88EE899E8A4E8AFE8BAE8C5E8D0EC
:106C1C00E8DBE8E6E8F1E8FCE907E912E91DE92818
:106C2C00E933E93EE949E954E95FE96AE975E98044
:106C3C00E98CE997E9A2E9ADE9B8E9C3E9CEE9D96C
:106C4C00E9E4E9EFE9FAEA05EA10EA1BEA26EA3197
:106C5C00EA3CEA47EA52EA5DEA68EA73EA7EEA89C4
:106C6C00EA94EA9FEAAAEAB5EAC0EACBEAD6EAE1F4
:106C7C00EAECEAF8EB03EB0EEB19EB24EB2FEB3A17
:106C8C00EB45EB50EB5BEB66EB71EB7CEB87EB9244
:106C9C00EB9DEBA8EBB3EBBEEBC9EBD4EBDFEBEA74
:106CAC00EBF5EC00EC0BEC16EC21EC2CEC37EC429D
:106CBC00EC4DEC59EC64EC6FEC7AEC85EC90EC9BC5
:106CCC00ECA6ECB1ECBCECC7ECD2ECDDECE8ECF3F4
:106CDC00ECFEED09ED14ED1FED2AED35ED40ED4B1D
:106CEC00ED56ED61ED6CED77ED82ED8DED98EDA34C
:106CFC00EDAEEDB9EDC5EDD0EDDBEDE6EDF1EDFC76
:106D0C00EE07EE12EE1DEE28EE33EE3EEE49EE549B
:106D1C00EE5FEE6AEE75EE80EE8BEE96EEA1EEACCB
:106D2C00EEB7EEC2EECDEED8EEE3EEEEEEF9EF04FA
:106D3C00EF0FEF1AEF25EF31EF3CEF47EF52EF5D1E
:106D4C00EF68EF73EF7EEF89EF94EF9FEFAAEFB54B
:106D5C00EFC0EFCBEFD6EFE1EFECEFF7F002F00D79
:106D6C00F018F023F02EF039F044F04FF05AF065A3
:106D7C00F070F07BF086F092F09DF0A8F0B3F0BECE
:106D8C00F0C9F0D4F0DFF0EAF0F5F100F10BF116F8
:106D9C00F121F12CF137F142F14DF158F163F16E23
:106DAC00F179F184F18FF19AF1A5F1B0F1BBF1C653
:106DBC00F1D1F1DCF1E7F1F2F1FEF209F214F21F7C
:106DCC00F22AF235F240F24BF256F261F26CF277A3
:106DDC00F282F28DF298F2A3F2AEF2B9F2C4F2CFD3
:106DEC00F2DAF2E5F2F0F2FBF306F311F31CF327FF
:106DFC00F332F33DF348F353F35FF36AF375F38027
:106E0C00F38BF396F3A1F3ACF3B7F3C2F3CDF3D852
:106E1C00F3E3F3EEF3F9F404F40FF41AF425F4307D
:106E2C00F43BF446F451F45CF467F472F47DF488AA
:106E3C00F493F49EF4A9F4B4F4BFF4CBF4D6F4E1D7
:106E4C00F4ECF4F7F502F50DF518F523F52EF539FC
:106E5C00F544F54FF55AF565F570F57BF586F5912A
:106E6C00F59CF5A7F5B2F5BDF5C8F5D3F5DEF5E95A
:106E7C00F5F4F5FFF60AF615F620F62BF637F64282
:106E8C00F64DF658F663F66EF679F684F68FF69AAA
:106E9C00F6A5F6B0F6BBF6C6F6D1F6DCF6E7F6F2DA
:106EAC00F6FDF708F713F71EF729F734F73FF74A03
:106EBC00F755F760F76BF776F781F78CF798F7A330
:106ECC00F7AEF7B9F7C4F7CFF7DAF7E5F7F0F7FB5A
:106EDC00F806F811F81CF827F832F83DF848F85382
:106EEC00F85EF869F874F87FF88AF895F8A0F8ABB2
:106EFC00F8B6F8C1F8CCF8D7F8E2F8EDF8F8F904E0
:106F0C00F90FF91AF925F930F93BF946F951F95C01
:106F1C00F967F972F97DF988F993F99EF9A9F9B431
:106F2C00F9BFF9CAF9D5F9E0F9EBF9F6FA01FA0C5F
:106F3C00FA17FA22FA2DFA38FA43FA4EFA59FA6588
:106F4C00FA70FA7BFA86FA91FA9CFAA7FAB2FABDB1
:106F5C00FAC8FAD3FADEFAE9FAF4FAFFFB0AFB15DF
:106F6C00FB20FB2BFB36FB41FB4CFB57FB62FB6D09
:106F7C00FB78FB83FB8EFB99FBA4FBAFFBBAFBC539
:106F8C00FBD1FBDCFBE7FBF2FBFDFC08FC13FC1E5E
:106F9C00FC29FC34FC3FFC4AFC55FC60FC6BFC7689
:106FAC00FC81FC8CFC97FCA2FCADFCB8FCC3FCCEB9
:106FBC00FCD9FCE4FCEFFCFAFD05FD10FD1BFD26E5
:106FCC00FD32FD3DFD48FD53FD5EFD69FD74FD7F09
:106FDC00FD8AFD95FDA0FDABFDB6FDC1FDCCFDD739
:106FEC00FDE2FDEDFDF8FE03FE0EFE19FE24FE2F64
:106FFC00FE3AFE45FE50FE5BFE66FE71FE7CFE8791
:10700C00FE92FE9EFEA9FEB4FEBFFECAFED5FEE0B9
:10701C00FEEBFEF6FF01FF0CFF17FF22FF2DFF38E2
:10702C00FF43FF4EFF59FF64FF6FFF7AFF85FF9010
:10703C00FF9BFFA6FFB1FFBCFFC7FFD2FFDDFFE840
:0F704C00FFF3FFFE3031323334353637040201A3
:10409A00C100C10141004800C10241004900680055
:1040AA000064000000010001000200020003000495
:1040BA0000040005000500060006000700080008C5
:1040CA0000090009000A000B000B000C000C000D8F
:1040DA00000D000E000F000F00100010001100125A
:1040EA000012001300130014001500150016001624
:1040FA0000170017001800190019001A001A001BEF
:10410A00001C001C001D001D001E001E001F0020B8
:10411A000020002100210022002300230024002483
:10412A00002500260026002700270028002800294D
:10413A00002A002A002B002B002C002D002D002E17
:10414A00002E002F002F00300031003100320032E3
:10415A0000330034003400350035003600360037AD
:10416A000038003800390039003A003B003B003C77
:10417A00003C003D003E003E003F003F0040004042
:10418A00004100420042004300430044004500450C
:10419A000046004600470047004800490049004AD7
:1041AA00004A004B004C004C004D004D004E004FA1
:1041BA00004F00500050005100510052005300536C
:1041CA000054005400550056005600570057005836
:1041DA0000580059005A005A005B005B005C005D01
:1041EA00005D005E005E005F0060006000610061CB
:1041FA000062006200630064006400650065006696
:10420A00006700670068006800690069006A006B5F
:10421A00006B006C006C006D006E006E006F006F2A
:10422A0000700071007100720072007300730074F4
:10423A0000750075007600760077007800780079BE
:10424A000079007A007A007B007C007C007D007D8A
:10425A00007E007F007F0080008000810081008254
:10426A00008300830084008400850086008600871E
:10427A000087008800890089008A008A008B008BE9
:10428A00008C008D008D008E008E008F00900090B3
:10429A00009100910092009200930094009400957E
:1042AA000095009600970097009800980099009A48
:1042BA00009A009B009B009C009C009D009E009E13
:1042CA00009F009F00A000A100A100A200A200A3DD
:1042DA0000A300A400A500A500A600A600A700A8A8
:1042EA0000A800A900A900AA00AB00AB00AC00AC72
:1042FA0000AD00AD00AE00AF00AF00B000B000B13D
:10430A0000B200B200B300B300B400B400B500B606
:10431A0000B600B700B700B800B900B900BA00BAD1
:10432A0000BB00BC00BC00BD00BD00BE00BE00BF9B
:10433A0000C000C000C100C100C200C300C300C465
:10434A0000C400C500C500C600C700C700C800C831
:10435A0000C900CA00CA00CB00CB00CC00CC00CDFB
:10436A0000CE00CE00CF00CF00D000D100D100D2C5
:10437A0000D200D300D400D400D500D500D600D690
:10438A0000D700D800D800D900D900DA00DB00DB5A
:10439A0000DC00DC00DD00DD00DE00DF00DF00E025
:1043AA0000E000E100E200E200E300E300E400E5EF
:1043BA0000E500E600E600E700E700E800E900E9BA
:1043CA0000EA00EA00EB00EC00EC00ED00ED00EE84
:1043DA0000EE00EF00F000F000F100F100F200F34F
:1043EA0000F300F400F400F500F600F600F700F719
:1043FA0000F800F800F900FA00FA00FB00FB00FCE4
:10440A0000FD00FD00FE00FE00FF00FF01000101AB
:10441A000101010201020103010401040105010570
:10442A000106010701070108010801090109010A3A
:10443A00010B010B010C010C010D010E010E010F04
:10444A00010F0110011001110112011201130113D0
:10445A00011401150115011601160117011701189A
:10446A0001190119011A011A011B011C011C011D64
:10447A00011D011E011F011F01200120012101212F
:10448A0001220123012301240124012501260126F9
:10449A0001270127012801280129012A012A012BC4
:1044AA00012B012C012D012E013001310132013382
:1044BA0001340135013701380139013A013B013C28
:1044CA00013E013F014001410142014301450146CC
:1044DA00014701480149014A014C014D014E014F72
:1044EA000150015201530154015501560157015916
:1044FA00015A015B015C015D015E016001610162BB
:10450A00016301640165016701680169016A016B60
:10451A00016C016E016F0170017101720173017505
:10452A000176017701780179017B017C017D017EA9
:10453A00017F01800182018301840185018601874F
:10454A000189018A018B018C018D018E01900191F3
:10455A000192019301940195019701980199019A99
:10456A00019B019D019E019F01A001A101A201A43D
:10457A0001A501A601A701A801A901AB01AC01ADE2
:10458A0001AE01AF01B001B201B301B401B501B688
:10459A0001B701B901BA01BB01BC01BD01BE01C02D
:1045AA0001C101C201C301C401C601C701C801C9D1
:1045BA0001CA01CB01CD01CE01CF01D001D101D277
:1045CA0001D401D501D601D701D801D901DB01DC1B
:1045DA0001DD01DE01DF01E001E201E301E401E5C1
:1045EA0001E601E801E901EA01EB01EC01ED01EF65
:1045FA0001F001F101F201F301F401F601F701F80A
:10460A0001F901FA01FB01FD01FE01FF02000201AD
:10461A000202020402050206020702080209020B4C
:10462A00020C020D020E020F0211021202130214F0
:10463A000215021602180219021A021B021C021D96
:10464A00021F02200221022202230224022602273A
:10465A0002280229022A022B022D022E022F0230E0
:10466A000231023302340235023602370238023A84
:10467A00023B023C023D023E023F02410242024329
:10468A0002440245024602480249024A024B024CCF
:10469A00024D024F02500251025202530254025674
:1046AA000257025A025C025F0261026302660268F2
:1046BA00026A026D026F0272027402760279027B4A
:1046CA00027D02800282028402870289028B028EA4
:1046DA0002900292029502970299029C029E02A1FE
:1046EA0002A302A502A802AA02AC02AF02B102B357
:1046FA0002B602B802BA02BD02BF02C102C402C6B1
:10470A0002C902CB02CD02D002D202D402D702D908
:10471A0002DB02DE02E002E202E502E702E902EC63
:10472A0002EE02F102F302F502F802FA02FC02FFBB
:10473A000301030303060308030A030D030F03110E
:10474A00031403160318031B031D03200322032467
:10475A0003270329032B032E0330033203350337C0
:10476A000339033C033E0340034303450348034A1A
:10477A00034C034F0351035303560358035A035D73
:10478A00035F0361036403660368036B036D036FCE
:10479A000372037403770379037B037E0380038226
:1047AA0003850387038C03900395039A039F03A34E
:1047BA0003A803AD03B103B603BB03BF03C403C914
:1047CA0003CE03D203D703DC03E003E503EA03EED7
:1047DA0003F303F803FD04010406040B040F041495
:1047EA000419041E04220427042C04300435043A54
:1047FA00043E04430448044D04510456045B045F18
:10480A0004640469046D04720477047C04800485DA
:10481A00048A048E04930498049C04A104A604AB9D
:10482A0004AF04B404BD04C704D004DA04E304ECFE
:10483A0004F604FF05090512051B0525052E053892
:10484A000541054B0554055D05670570057A058325
:10485A00058C0596059F05A905B205BB05C505CEBC
:10486A0005D805E10734088609D90B2B0C7E0DD033
:10487A000F23107511C8131A146D15C01712186575
:10488A0019B71B0A1C5C1DAF1F01205421A722F96E
:10489A00244C259E26F1284329962AE82C3B2D8D67
:1048AA002EE041086400410865004108660042089C
:1048BA006700004108690042086A000041000000E0
:1048CA004100010141086C0041086D0041086E0079
:1048DA0042000200004200040000420006000042BA
:1048EA000008000042000A000042000C00004108D3
:1048FA006F004108708041087180420872000041CF
:10490A0008740041087580410876804208770000E3
:10763E00E47F587E1BFDFC900CE9E0F8A3A3A3E0C9
:10764E00127219900CED12735D7BFF7A03900CEDA4
:10765E00E0FCA3E0FDA3E0FEA3E0FFE4F9F8128B4B
:10766E0069900CED12735D900CEDE0FCA3E0FDA3B0
:10767E00E0FEA3E0227E10E4FF900CE9FDFCE0F8B2
:10768E00A3E0F9A3E0FAA3E0FB2278EB7C0D7D01E9
:10769E007B017E007F0202712B900D4E7B017A0DD5
:1076AE00793BEBF0A3EAF0A3E9F0227FF47E01E44C
:1076BE00FDFC900CE9E0F8A3A3A3E0027219E4909C
:1076CE000DE9F0A3F078EB7C0D7D017B012225E026
:1076DE00FFE033FE744C2FF58274003EF583ECF020
:1076EE00A3EDF0227A08FFE4FBF9F8D302733624F7
:1076FE003CFFEE34F6FEED34FFFDEC34FFFC229041
:10770E000004E0FEA3E0FFD32290000512718CFF6F
:10771E0090000612718CFD90000402718CFFE47BC8
:10772E0064FAF9F81272A4900CF112735DE47FFF03
:10773E007EFFFDFC900CF122FFEB2FFFEA3EFEE9EF
:10774E003DFDE83CFC02735D900E0874FFF5F012EF
:10775E007203FAD3E5F09400EA94002278E97C0DE6
:10776E007D017B0122900CE8E0900CE725E0FFE024
:10777E0033FE2290000312718CFF22900E08E4F06B
:10778E00A37410F022D3EF94D3EE940322D3EF948C
:10779E0033EE940A22FDE0FF3395E0FEEF25E0FF85
:1077AE00EE33FE22900CED02735D127219900CF105
:1077BE0012735D900CF122900CF1A3A3E0FEA3E0F6
:1077CE00FDAC0622FE7F0202712B900873E094D06E
:1077DE00900872E0940022900878E094C0900877A8
:1077EE00E09400223EF583E0FEA3E0FFE4FCFD22E0
:1077FE00D3EF94F4EE940022FF900CE912735D9097
:10780E000CE922FFE4FB7A08F9F8028B69E004F038
:04781E00C36480229D
:108F3600E4F584758810758902758E02758A017547
:068F46008C0143A8022289
:0D8F7100E4F584759A4075F809759D30226D
:108D8600E4F58475E880900864E0F5BB75840275A7
:108D9600BCF975E880A3E0F5BBE4F58443E712224D
:078FD000E4F58475D10222D3
:108EA40075840F75A4CF75AD0175A50175A67F7581
:098EB400A77F75E10375E340227C
:108AD700E4FFFE75840F438A0353A1DFF58475B75E
:108AE7003075840F43A120438901758D01758F016E
:108AF700758E040FBF00010EEF640F4E70F54389AA
:108B070002E58920E4130FBF00010EBE0FF3BFFF7C
:0C8B1700F0E4F58443EF1080E87597024D
:018B2300222F
:108DE500128AD7128EA4128F36128F71128FD0125B
:0E8DF5008D86900047E0FF128F7E43F602222B
:06503300E4900866F02283
:078FD7009008667401F0220E
:107B96007B017A0D793B128CCBEF7003027CE3906C
:107BA6000D3DE012739A7C0E047C2E057BDE147B61
:107BB600CB167BD6177BE31A7BF71B7C021D7C0852
:107BC6001E00007C579000487401F0C209027C57E1
:107BD600E4900048F0027C57D202027C57900D4B8D
:107BE6001276AA127173FE900047E0FF6E706280F3
:107BF60005900047E0FF128F1F027C57128FD702B5
:107C06007C57125033027C571276A7127781900068
:107C160047E06F703CA3E06030900D4E1276B012D4
:107C26007717FB12885D80211276A7127781900064
:107C360047E06F701CA3E06010900D4E1276B012F4
:107C46007717FB1286E4128DA6900047E0FF128E8E
:107C5600EF900048E07003027B96900D3DE01460C3
:107C66001B24FA602314605524066003027B9612D7
:107C76007CE4900D12F0128FF0027CDD127CE49011
:107C86000D12F0128DA6804F127CFF900D511276C8
:107C9600B0127781127725FD90000512718CFBC01A
:107CA60003900D51E0FBA3E0FAA3E0F99000061261
:107CB600718C900D77F0D00312848B801A127CFFA2
:107CC600900D511276B0127781127725FD9000053E
:0D7CD60012718CFB127E60128F97027B965C
:107CE3002212501B7B017A0D793B900D4BEBF0A3D5
:107CF300EAF0A3E9F090000312718C2212501B7B6F
:067D0300017A0D793B221C
:1089890075FFDE75FFAD9000477463F0128DE5D277
:10899900AF128E8A128DA6AF84E4F5848F8490007D
:1089A90049E06008128FF0E4900049F0300010901F
:1089B9000047E0FF7BFF7A50793C124FA9C2003093
:1089C9000110900866E07008900047E0FF128ED60B
:0789D900C201127B9680C071
:0350060002494D0F
:10494D00C0E0C0F0C083C082C0D075D000C000C030
:0D495D0001C002C003C004C005C006C007B1
:10496A0090086BE004F0700690086AE004F0C390C7
:10497A00086BE0940490086AE094005003024D5ECC
:10498A0090086AE4F0A3F0900CE1740FF0A374FFAE
:10499A00F0A37408F0A37420F0900869E014600F83
:1049AA0014601114603924037038125001803312D4
:1049BA008FB7802E900867E4F0A3F01279EF900881
:1049CA0068E004F07006900867E004F0C390086895
:1049DA00E09408900867E06480948040DE800312C7
:1049EA008F4C90086912781B94844002E4F0900C72
:1049FA00E3E0FEA3E0FF900CE1E0FCA3E0FD12730C
:104A0A00F1900CDD12735D900869E0FF75F00212F7
:0A4A1A007151AFF0EF7003024D5E22
:074A2400900CE7E4F0A3F0A1
:104A2B0012777374442FF974503EFA900D0574FF8E
:104A3B001276B1900D05E0FBA3E0FAA3E0F9127139
:104A4B0073FD540FFB900D08E4F0A3EBF0EDC45491
:104A5B000FFDA3E4F0A3EDF0900D05E0FB9000013A
:104A6B0012718C540FFD900D0CE4F0A3EDF0741348
:104A7B002FF582740D1277F2900D0E12735D900C60
:104A8B00E7E0FEA3E0FF4E6006EF64054E70139067
:104A9B000D09E0900D0812777A74272FF5827400B8
:104AAB00800A127773741D2FF582740D1277F290B2
:104ABB000CFD12735D900CFD12768CC374FF9BFF83
:104ACB00740F9AFEE499FDE498FCA312735D900DAC
:104ADB000E127678FFE4FBFAF9F8D312734C5032CE
:104AEB00E47FAA7E02900D0E12768AC312734C508D
:104AFB00217F607EF07DFF7CFF900D0E1276C3123E
:104B0B0077B27BAA7A0212765B2428FFEE3423025B
:104B1B004B63900D0E127678FFE47BAA7A02F9F8BC
:104B2B00D312734C503CE4FF7E10FDFC900D0E1223
:104B3B00768CC312734C502A7F787EEC7DFF7CFF02
:104B4B00900D0E1276C312766FFFE47B567A0D1220
:104B5B00766A246FFFEE3417FEE43DFDE43CFC1255
:104B6B0077B2127675FF900CF5127672FF900CF9F6
:104B7B0012735D900CFD127678127806127678FF20
:104B8B00E4FBFA1276F750177E08127685C3127380
:104B9B0036500C1276B912766F127811024BFC90CC
:104BAB000CE91276781276F25025E4FF7E0C127621
:104BBB0087C312733650187FDC7E051276BD1276D2
:104BCB006FFFE4FB7A0412766A1276FD024BFC90BF
:104BDB000CE91276787A0C1276F45018127683C39D
:104BEB00127336500F12763E24B3FFEE34B51277A4
:104BFB00031277B2900CF512768C127675900CF539
:104C0B00127746900D01127678127806127678FF9D
:104C1B00E4FBFA1276F75019E4FF7E08127687C38D
:104C2B00127336500C1276B912766F127811024C41
:104C3B0092900CE91276781276F25026E4FF7E0CF5
:104C4B00127687C31273365019E47FDC7E05127619
:104C5B00BE12766FFFE4FB7A0412766A1276FD02BF
:104C6B004C92900CE9127678FFE4FB7A0C1276F7F3
:104C7B005018127683C3127336500F12763E24B33C
:104C8B00FFEE34B51277031277B2900CF912768CD3
:104C9B00127675900CF9127746E47F167E03FDFCB5
:104CAB00900CF512768C1277B812767812772B124D
:104CBB00768CD312734C400A900CF112736900007E
:104CCB00FFFF1277C5900D0BE0900D0A1276DCE416
:104CDB007F167E03FDFC900CF912768C1277B812BE
:104CEB00767812772B12768CD312734C400A900C79
:104CFB00F11273690000FFFF1277C5900D0DE09064
:054D0B000D0C1276DC26
:104D1000900CE8E004F07006900CE7E004F0900CD2
:104D2000E7E07004A3E064066003024A2B78E57CA8
:104D30000C7D017B017A0079601276A078607C009E
:104D40007D017B017A0079627E007F0212712B78EF
:0E4D5000627C007D017B017A0C79E51276A071
:104D5E00D007D006D005D004D003D002D001D000A9
:0B4D6E00D0D0D082D083D0F0D0E03253
:0450010043E810224E
:098FB700758402D2ECE4F5842279
:1079EF00900867E0FEA3E0FFEE6003027AC6EFB4F3
:1079FF0008004003027AC6907A0DF8282873027A9D
:107A0F0025027A3C027A53027A6D027A86027A95BF
:107A1F00027AA4027AB312776A7A00795C1276A09E
:107A2F007A00794C127698907050027AC012776A69
:107A3F007A00795E1276A07A00794E12769890705D
:107A4F0051027AC012776A7A0079601276A01276A4
:107A5F00D37A0079501276A0907052027AC01277C2
:107A6F006A7A0079621276A01276D37A007952126E
:107A7F0076A0907053803A1276CC7A0079541277B0
:107A8F00D2907054802B1276CC7A0079561277D21E
:107A9F00907055801C1276CC7A0079581277D2905C
:107AAF007056800D1276CC7A00795A1277D2907078
:107ABF0057E493900DE8F0E4F584C2FA900000E0EB
:107ACF00F59B30FFFDC2FFE4FFFE0FBF00010EEF7D
:107ADF0064324E70F5900DE8E0F59B30FFFDC2FF6C
:107AEF00E4FEFF0FBF00010EEF64324E70F5900DF4
:107AFF00E9E0F59B30FFFDC2FFE4FEFF0FBF000181
:107B0F000EEF64324E70F5900DEAE0F59B30FFFDFD
:107B1F00C2FFE4FEFF0FBF00010EEF64324E70F59F
:107B2F00900000E0F59B30FFFDC2FFE4FEFF0FBFAA
:107B3F0000010EEF64324E70F5900DE8E0F59B30CA
:107B4F00FFFDC2FFE4FEFF0FBF00010EEF64324ED8
:107B5F0070F5900DEBE0F59B30FFFDC2FFE4FEFFEB
:107B6F000FBF00010EEF64324E70F5900DECE0F593
:107B7F009B30FFFDC2FFE4FEFF0FBF00010EEF645D
:067B8F00324E70F5D2FA3F
:017B950022CD
:0350300002744ABD
:10744A00C0E0C0F0C083C082C0D075D000C000C008
:0D745A0001C002C003C004C005C006C00789
:1074670053E8DFAFBFEFFEADBE7C00E42DFFEC3E7F
:10747700900024F0A3EFF0900024E0FCA3E0900834
:10748700641277A374272FF58274001276E99008A7
:107497006412781B948850030275FDE4F090003164
:1074A700E0FFA3E0900010CFF0A3EFF090002FE0F3
:1074B700FFA3E0900012CFF0A3EFF090002DE0FFC4
:1074C700A3E0900014CFF0A3EFF090002BE0FFA310
:1074D700E0900016CFF0A3EFF0900029E0FFA3E0C3
:1074E700900018CFF0A3EFF0900027E0FFA3E09003
:1074F700001ACFF0A3EFF090003FE0FFA3E0900069
:107507001CCFF0A3EFF0900041E0FFA3E090001E36
:10751700CFF0A3EFF0900043E0FFA3E0900020CF6F
:10752700F0A3EFF0900045E0FFA3E0900022CFF03A
:10753700A3EFF0900001E06033E4FFEF25E02410B3
:10754700F582E43400F583E0FCA3E0FDEF25E024B9
:1075570054F582E4340D1276EA0FEFB40ADD900099
:1075670001E004F0E0D3940F4002E4F0900001E062
:1075770070047D0180027D007F0012761E70047DFD
:107587000180027D007F0112761E70047D0180025A
:107597007D007F0212762670047D0180027D007FC8
:1075A7000312762670047D0180027D007F04127627
:1075B7002E70047D0180027D007F0512762E7004F7
:1075C7007D0180027D007F0612763670047D018082
:1075D700027D007F0712763670047D0180027D00F0
:1075E7007F08127822900001E070047D0180027DFF
:0C75F700007F09127822900864E0F5BBC8
:10760300D007D006D005D004D003D002D001D000DB
:10761300D0D0D082D083D0F0D0E032127822900044
:1076230001E022127822900001E0221278229000D9
:0B76330001E022127822900001E0220A
:035039000288CC1E
:1088CC00C0E0C0F0C083C082C0D075D000C005C06D
:1088DC0006C007758402C2ED900026E5BEF0E07577
:1088EC00F010A49008651277A374372FF5827400EA
:1088FC003EF583E5F0F0A3EDF090086512781B943B
:10890C00884002E4F0900865E0F5BB758400D00760
:0F891C00D006D005D0D0D082D083D0F0D0E032BA
:10865B00900039A3E0FEC394F040047F108016EE27
:10866B00C3944040047F20800CEED3942040047FC1
:10867B00408002E4FF90086DE033333354F8FEA3DF
:10868B00E0907058934EFE900048E0C4333333545F
:06869B00804E4FFEC2906C
:1086A100127789900E0874FFF5F0127203FCD3E57E
:0886B100F09400EC940050EB82
:1086B900E4FDEEA805088002C313D8FC139286C214
:0186C9008729
:0886CA0012778912775650FB6C
:0286D200D2874D
:0886D40012778912775650FB62
:0786DC000DEDB408DAD290A5
:0186E3002274
:104D790090003BE0FFA3E0900002CFF0A3EFF0909A
:104D8900003DE0FEA3E0FF900004EEF0A3EFF0D3B6
:104D9900900007E09F900006E09E5016900004E006
:104DA900FFA3E0A3CFF0A3EFF090000AE4F0A3740F
:104DB90080F0900008E0FEA3E0FF900002E0FCA371
:104DC900E0FDC39FEC9E4011900008ECF0A3EDF0CC
:104DD90090000CE4F0A37480F012770D94A3EE9484
:104DE900004003D38001C392B01277FE4003D38001
:104DF90001C392B112770D943BEE94024003D38024
:104E090001C392B21277934003D38001C392B312C4
:104E1900770D94BCEE94054003D38001C392B4127C
:104E2900779B4003D38001C392B5D3900005E094EA
:104E39004C900004E0940F4003D38001C392B6D391
:104E490090000BE0940090000AE09400406190000B
:104E590006127710944CEE940F4004D2B68040129B
:104E6900779B4004D2B58037D3EF94BCEE940540CC
:104E790004D2B4802A1277934004D2B38021D3EFAD
:104E8900943BEE94024004D2B280141277FE40049F
:104E9900D2B1800BD3EF94A3EE94004002D2B0902C
:104EA900000BE024FFF090000AE034FFF08007E4F3
:104EB900900006F0A3F0D3ED94A3EC94004003D343
:104EC9008001C392A0D3ED94F4EC94004003D38005
:104ED90001C392A1900002127710943BEE94024014
:104EE90003D38001C392A21277934003D38001C3F5
:104EF90092A390000212771094BCEE94054003D35C
:104F09008001C392A412779B4003D38001C392A569
:104F1900D3900003E0944C900002E0940F4003D337
:104F29008001C392A6D390000DE0940090000CE09C
:104F390094004061900008127710944CEE940F4051
:104F490004D2A6804012779B4004D2A58037D3EFC4
:104F590094BCEE94054004D2A4802A1277934004AD
:104F6900D2A38021D3EF943BEE94024004D2A280D5
:104F7900141277FE4004D2A1800BD3EF94A3EE94D0
:104F8900004002D2A090000DE024FFF090000CE058
:0F4F990034FFF08007E4900008F0A3F012865B6D
:014FA80022E6
:0F50090090086EE004F0E0D394024002E4F0223D
:088FC00090086DE06401F0224D
:10830B00900870E0A3F0E5B05480900870F0A3E003
:10831B00FD900870E0FE6D90000EF0EE702EED609B
:10832B0007E4900872F0A3F0900873E004F0700675
:10833B00900872E004F0D31277D8403C90086FE0BD
:10834B007002D20090086F7401F0802C900871E0DD
:10835B007026C31277D8501B300209900048E06496
:10836B0001F0800F900048E06009A37401F0E490E5
:10837B000048F0E490086FF0900875E0A3F0E5A0DA
:10838B005480900875F0A3E0FD900875E0FE6D90A9
:10839B00000FF0EE702EED6007E4900877F0A3F07D
:1083AB00900878E004F07006900877E004F0D312A0
:1083BB0077E54024900874E07003128FC090087426
:1083CB007401F022900876E0700EC31277E550032B
:0883DB00125009E4900874F04F
:0183E3002277
:108F4C0090086CE0700512830B8003124D79900829
:068F5C006CE06401F0224C
:108DC600E0FEA3E0A60608F6E4F584C2AF43B701C9
:0F8DD60022E475F001027203EEF0A3EFF0A32286
:108C2A00AB84A2AF9206E4FCFDED900DED12735DEC
:108C3A00900DEF780E128DC6438F02438F0118E60E
:108C4A00FE08E6F5828E83E4F053B7FEF58FA2069E
:068C5A0092AFAF038F840E
:018C600022F1
:028BAD00AB0516
:108BAF00AA84A2AF9207E4FCFDED900DF112735D64
:108BBF00EBFF3395E0FEEFF44E601C900DF3781051
:108BCF00128DC6758F0118E6FC08E6F5828C83EBD3
:0F8BDF00F053B7FEE4F58FA20792AFAF028F8479
:018BEE002264
:10892B00900DD6128DDEECF0A3EDF0A3EAF0A3EBE5
:10893B00F0900DDAE07002A3E06042900DD6E0FEFD
:10894B00A3E0FFA3E0FCA3E0F5828C83E0FD128B98
:10895B00AD900DDBE024FFF0900DDAE034FFF090EA
:10896B000DD9E004F07006900DD8E004F0900DD70F
:0E897B00E004F070BC900DD6E004F080B42251
:088FC800E4900C79F0A3F02203
:108CF700900C79E0FEA3E0FF128C2A900C79E0FE3D
:108D0700A3E0FF7C087D797B007A0412892BE4902D
:068D17000C79F0A3F0222C
:0A876D00A905900DDCEEF0A3EFF07B
:10877700EE54FCFE900C79E0FCA3E0FD7002EE6C79
:10878700604CED4C6003128CF7900DDCE0FEEE546C
:10879700FCFE7F00900C79F0A3EFF0900DDE128DB8
:1087A700DE7408F0A37479F07E04900DDE128DD785
:1087B70085F082F583E493FD900DE0128DD785F067
:1087C70082F583EDF0EF1F70011EEF4E70DC900D08
:1087D700DCE0FCA3E0FDEC5403FC74792DF5827416
:0687E700083CF583E9F0F7
:0187ED002269
:108BEF00900DC1128DDEEBF0A3EAF0A3E9F0900D2A
:108BFF00C674FFF5F012720345F0601E900DC1129E
:108C0F008DD7AFF0FE900DC3E0FBA3128DD7A9F067
:0B8C1F00FA127173FD12876D80D422E1
:10491A00420C7E0000420C830000420C850000C15C
:05492A0004C105C103FA
:108A8800900C85E475F0011271EDFCE5F064404C42
:108A980022D3900C7FE09400900C7EE06480948058
:108AA80022E0FEA3E02487F582740C22E0FBA3E019
:108AB800FAA3E0F98E8275830022900C85F0A3F06A
:0F8AC80022900C82E004F022900C81E004F02256
:0A8FAD00C205C204E4900CC7F022D4
:108D4200E4900C7EF0A3F0900C83F0A3F0900C87DB
:108D5200F0128AC2900C81F0A37440F0E4900C806F
:028D6200F022FD
:068FDE00128FAD028D426E
:108EBD00E4F5848FC343C30175C04475CF8EC2C31F
:098ECD0043E602900C7C04F02243
:10501B00E4F58420C7FDC2C2128FDEE4900C7CF055
:01502B002262
:0B8F9700E4F584D2C2900C7C04F022B0
:0D8F7E00AE07128EBD900C7DEFF0028FDE6D
:108D1D00E4900E0AF0A3F0300502FF222004FDD2EC
:108D2D0005900CC8E4F0A37410F0900CCBEFF0E4B8
:048D3D00A3F07F011F
:018D4100220F
:108C970030050A900CC8E07002A3E070037F002241
:108CA700900CC9E024FFF0900CC8E034FFF0900C62
:108CB700CCE0FE04F074CD2EF582E4340CF583EF9E
:048CC700F07F012217
:0B8FA200300507C205D204128F6222C6
:0E8F6200AF84E4F58420C7FDC2C4D2C58F845D
:018F700022DE
:1087EE00900DC9EBF0A3EAF0A3E9F0900C7CE070D9
:1087FE0002FF22900DCCE0FE6005D3941040037F63
:08880E000022128D1DEF6044F1
:10881600E4900DCEF0900DCCE0FF900DCEE0FEC3BF
:108826009F501A900DC9128AB412718CFF128C9740
:10883600EF7002FF22900DCEE004F080D8E4900C99
:10884600C7F0128FA2900DCDE070032004FD900CAE
:04885600C7E0FF2256
:03885A007FFF227B
:0E83E400900DF5EBF0A3EAF0A3E9F0A3EDF0A5
:1083F200E4FF128A9950012253E6FD900C85128AFD
:10840200A93EF583E0FF128A887003128AC2128A9B
:10841200C97003128AD0E4FE900DF8E0FDEEC39D10
:10842200502FEEC39F502A900C85E0FC128AAB3C81
:10843200F583E0FD900DF5128AB4ED1271CB128A2C
:10844200887003128AC2128AC97003128AD00E80FF
:10845200C7EEC39F5013128A887003128AC2128A0F
:10846200C97003128AD00E80E8900C7FE024FFF0DE
:10847200900C7EE034FFF043E602900DF8E0FEEF50
:08848200C39E50028002AF0608
:01848A0022CF
:0C8F8B00128A9940047F0180027F0022BE
:03501800027D090D
:107D0900C0E0C0F0C083C082C0D075D000C000C040
:037D190006C0079A
:107D1C00C208AFC1EF12739A7D52087D52107D627A
:107D2C00187D67207D74287DA1307DAC387DB460D2
:107D3C007DAF687DB4707DAF787DBC807DBC907E5E
:107D4C002CA000007E3A900CCBE0F5C2C2C5900C82
:107D5C00CAE4F0027E3C900CCC8028900CC774FDD9
:107D6C00F0D2C4D2C5027E3C900CCCE0FF900CCA81
:107D7C00E0C39F5014E0FF04F074CD2FF582E4347F
:107D8C000CF583E0F5C2027E3CD2C4900CC7E4F043
:107D9C00C204027E3CD2C5900CC774FEF0027E3C3D
:107DAC00027E31D203027E3C900C7BE4F0027E3CDE
:107DBC00900C7BE07020E5C2F0E0FFC3900C82E0F9
:107DCC009F7480F8900C81E06480985003128D426F
:107DDC00900C7BE004F0900C82E024FFF0900C817E
:107DEC00E034FFF0900C83128AA93EF583E5C2F0D3
:107DFC00900C83E475F0011271EDFEE5F064404ED9
:107E0C007006900C83F0A3F0900C7BE014F07020C3
:107E1C00900C7FE004F07018900C7EE004F0801061
:107E2C0030030DC203900CCAE4F0D2C58002D20814
:107E3C0030080EC2C6D2C6C2C5C2C4D2C2C208C2A3
:037E4C0004C2C3AA
:107E4F00D007D006D000D0D0D082D083D0F0D0E0F1
:017E5F0032F0
:058FE400A2C7E433FF09
:018FE9002265
:108A3600EFF0A3ECF0A3EDF0A3EBF0A3EAF0A3E9CB
:108A4600F0227403F0A374E8F0A3E584F0E4F5845F
:108A560022D2C4D2C5D2C2C2C3E4900E0FF0FF2206
:108A6600E0FBA3E475F001127203A9F0FA22E025F7
:108A7600E044A0F5C27F032274FFF5F01271ED45C4
:028A8600F022DC
:068FEA00C2C253E6FD22A5
:0681FB00900D68128A36A7
:10820100900D71128A4820C7FDC2C4D2C2D2C5E402
:10821100FF900E0FF030C3FDAEC1EE24F8602324B1
:10822100F8601F24F8602924F8603024F8603424B1
:10823100F870030282BE24F870030282C624380259
:1082410082CEEF7006900D68128A74C2C50282D484
:10825100900D69E0F5C27F050282D4900E0F740380
:10826100F08070EFB4050B900D69A3E0F5C27F06B5
:108271008061EF64067034900D70E0900D6B7005B5
:10828100128A668008E0FBA3E0FAA3E0F912717399
:10829100F5C2900D6FE024FFF0900D6EE034FFF019
:1082A100E07002A3E0702C7F078028EFB40706D2AC
:1082B100C47F09801E900E0F7405F08016900E0F7A
:1082C1007404F0800E900E0F7406F08006900E0F6D
:1082D1007401F0EFB40904C2C38025900E0FE0B41D
:1082E100030B900D71128A7E6003128A57900E0F54
:1082F100E06008C2C5D2C4C2C38005C2C3028216EF
:0983010020C7FD900D73E0F58426
:01830A002250
:0680D100900D80128A36BA
:1080D700900D88128A4820C7FDD2C2C2C4D2C5E417
:1080E700FF900E0FF030C3FDAEC1EE12739A811AE6
:1080F70000811D08811D10814218814D208155285E
:1081070081703081783881804081905081B85800E3
:1081170000811A0281BEC2C5EF7009900D80128AD4
:10812700740281C4EF640160030281C4900D80E092
:1081370025E044A1F5C27F040281C4900D81E0F5DA
:10814700C27F050281C4900E0F7403F0806FEFB4F5
:10815700050B900D81A3E0F5C27F068060EFB406A2
:1081670006D2C57F0180568018900E0F7404F080E8
:108177004C900E0F7406F08044EFB404047F028025
:108187003C900E0F7405F08034900D83128A66E5DB
:10819700C21271B9900D87E024FFF0900D86E0348C
:1081A700FFF0E07002A3E07004C2C280107F02807B
:1081B7000CD2C47F098006900E0F7401F0EFB4094A
:1081C70004C2C38025900E0FE0B4030B900D8812F4
:1081D7008A7E6003128A57900E0FE06008C2C5D2EC
:1081E700C4C2C38005C2C30280EC20C7FD900D8ABC
:0381F700E0F5842C
:0181FA002262
:107F9F00900DA0EFF0900DA3128A3F900DA1ECF081
:037FAF00A3EDF04F
:107FB200750A00543FF50B543F6058C37440950B4B
:107FC200FFE4950AFE900DA6E0FCA3E0FDC39FEC42
:107FD2009E50068C088D0980048E088F091280A39A
:107FE20060037F0222900DA2E02509F0900DA1E02E
:107FF2003508F0900DA8E0700B900DA4E5088509F6
:10800200F01271EDC3900DA7E09509F0900DA6E076
:108012009508F0900DA6E0F508A3E0F509D3E5096F
:108022009400E50894004076E5099440E508940040
:10803200500F1280A360037F0222E4F508F5098045
:10804200DC900DA0E0FFA3E0FCA3E0FDA3E0FBA316
:10805200E0FAA3E0F9900D6EE4F0A37440F0900D05
:10806200A8E0900D70F01281FB900E0FE060037F8C
:10807200022274C02509F50974FF3508F508900D30
:10808200A2E02440F0900DA1E03400F0900DA8E0B1
:10809200708B900DA475F0401271ED02801F7F006D
:1080A20022900DA0E0FFA3E0FCA3E0FDA3E0FBA370
:1080B200E0FAA3E0F9900D6EE508F0A3E509F0906F
:0F80C2000DA8E0900D70F01281FB900E0FE022E0
:108F0800900D86E4F0A304F01280D1900E0FE0607B
:078F1800037F01227F00220C
:108E3C00900E0EEBF07B017A0E790E900DA6E4F0FD
:0A8E4C00A304F0E4A3F0127F9F22BC
:108D6400C007900DAFE0FFA3E0900D86CFF0A3EF16
:108D7400F0D0071280D1900E0FE060037F01227FB4
:028D84000022CB
:108E5600C007900DB7E0FFA3E0900DA6CFF0A3EFFB
:0A8E6600F0E4A3F0D007127F9F2272
:108E70007B01E4900DE6F0227422F0A3EFF0A32230
:0A8E80007B01E4900DE6F07D042272
:0E8B2400900DE2EBF0A3EAF0A3E9F0A3EDF070
:108B3200E4900DE7F0900DE2E0FBA3E0FAA3E0F988
:108B4200A3E0900DCCF0900DE6E0900DCDF0E4FFA7
:108B52001287EEEFB4FF0D900DE7E0FE04F0EEC3D6
:068B6200940340D17E00E7
:018B680022EA
:0B8CCB00900E05EBF0A3EAF0A3E9F027
:108CD6007E007F007D1012741E900E05E0FBA3E05F
:108CE600FAA3E0F97D101283E4EF7002FF227F0100
:018CF600225B
:104FA900900D96128E787413F0127173900D99F01A
:104FB90090000112718C900D9AF090000212718C80
:104FC900900D9BF090000312718C900D9CF0900055
:104FD9000412718C900D9DF090000512718C900D4A
:104FE9009EF090000612718C900D9FF07A0D7996C3
:084FF900128E707D0A028B2468
:108ED600900DF9128E787403F0A374FFF07A0D7971
:098EE600F9128E707D04028B2448
:108F1F00900DFD128E78741CF0A374FFF07A0D790A
:078F2F00FD128E80028B246D
:108EEF00E4900E01F0A3EFF0A3740AF0A3EFF07A71
:098EFF000E7901128E80028B2411
:10492F00540D5400000000000000000000000000C3
:07493F000000000000000071
:1085C900E47F01FEFDFC1273E4E0F8A3E0F9A3E007
:1085D900FAA3E0FB229000061273E412735D900087
:1085E900121273E4E025E022F583E0FEA3E0FBC369
:1085F90074FF9BFF740F9EFEE49400FDE49400FC5D
:1086090022FEFDFC850C83850D82222454F582E42B
:10861900340DF583E0FEA3E0FF222413F582E43450
:108629000DF583EEF0A3EFF09000131273E4E0224E
:108639002410F582E4340022E47BFF7A0FF9F82252
:1086490090000A0273E4E0FCA3E0FDA3E0FEA3E0CE
:02865900FF22FE
:1078220090FFFF1273C0EDF090FFFF1273C0EFF0F4
:0678320090FFEE1273C08E
:1078380012860DE4F0A3F01285E7128614FBAA065F
:10784800E4F9F81285E712863912861BC3EF9BFF0D
:10785800EE9AFEE499FDE49812860CA3A312735DD8
:10786800E47F4012860AA3A31285D2C3127336405E
:107878000812860DE4F0A304F074FF7FC012860A94
:10788800A3A31285D2D3127336500812860D74FF43
:10789800F0A3F012860DE0FEA3E0FF4E700302791C
:0C78A800E9EFF47002EEF46003027933A3
:1078B4001285E7128614E4FCFD90000E1273E412A4
:1078C400735D90000E1285C9C3127336500D90007B
:1078D4000E1273E4127369000000011285E7241389
:1078E400F582E4340D12861BE4FCFD12864212720A
:1078F4001990000E1285CF128B691285DE1286391B
:1079040012861BE4FCFD9000061285CF1272191238
:10791400864912735D12864112864912864F128B74
:0C792400691285E712862370030279C403
:107930000279C112860DE0FEA3E064014E600302ED
:0279400079C408
:107942001285E72413F582E4340D1285F112864183
:107952001272191285DE2454F582E4340D1285F177
:1079620012864912735D90000A1285C9C3127336DA
:10797200500A128649127369000000019000061233
:1079820073E4C083C08212864F90000A1285CF1220
:107992008B69D082D0831285E41286391285F190E8
:1079A20000061285CF127219128641128B69C374B6
:1079B200FF9FFF740F9EFE1285E71286236003125B
:0279C2008E0332
:1079C4009000121273E4E0FF25E0128639F583E09B
:1079D400FCA3E0FDEF25E02454F582E4340DF583A7
:0579E400ECF0A3EDF042
:0679E9009000140273C0BF
:06494600410D1200C10941
:10853000900D92E075F014A42401F582E5F034F07A
:10854000AF8222FE7A0D79137B01900DC6E4F0A371
:108550007414F022AFF0FEE0FCA3E0F5828C83E41B
:1085600093FD22900D8EF0A3EFF0E4900D94F0A314
:10857000F022EF25E02413F582E4340DF583227513
:10858000F014A42401F974F035F0FA22EBF0AC07F2
:10859000A2AFE433A3F0C2AF22E475F0010272038C
:1085A000EDFFAD04EDCFF0A3EFF0E422F0900E105C
:1085B000E004F022900E10E0FFC322900D95E0043D
:0985C000F022900D94E004F02279
:1089E000128FC8E4900E10F01285B49406500B124A
:1089F0008572E4F0A31285AC80EE900E107406F040
:108A00001285B4940A500E1285727407F0A374FF95
:108A10001285AC80EBE4900E10F01285B4941E50D9
:108A20001275F014EF128537128543128BEF128501
:068A3000AD80E7028CF7A7
:108C6100900E0C7402F0E4A3F0128FC87EF07F0026
:108C71007A0E790C128C897EF27F597A0E790D1257
:088C81008C89128CF70289E0D6
:0E8C89007B01900DC6E4F0A304F0128BEF22E5
:108E030030020E20090B900048E06005D201D20920
:0D8E130022200208900048E0700204F022C6
:108E8A0090F259E493F4600990F000E4936402606C
:0A8E9A0003128C61E4900D12F02227
:108DA600900D12E0FFC3941E5015EF12857F7BFFD6
:108DB60078137C0D7D017E007F1412712BC209226F
:108E2000900D12E0C3941E5012128FC8900D1212B2
:0C8E30008533128543128BEF128CF72261
:068FF000128E20C20922CE
:08848B00900D75EDF0A3EBF07C
:10849300A3E004F0900D7AEFF0A3EBF0900D75E0FC
:1084A300FF900D7AE0FED39F506C75F014EE1285A9
:1084B30037900D7CF0A3EFF0900D7B128533900D78
:1084C3007EF0A3EFF0E4900D78F0A3F0900D7E1210
:1084D3008599900D7C12855412876D900D7DE00473
:1084E300F07006900D7CE004F0900D79E004F070DC
:1084F30006900D78E004F0C3900D79E09414900D8C
:1085030078E0940040C6128CF7900D7AE004F0A353
:10851300E004F002849F900D12E0FF900D76E0D30B
:0C8523009F5009A3E0C39F4003128DA6E7
:01852F002229
:0F7E6000900D8CEDF0900D8BEFF0900D8DEBF001
:107E6F00900D92EFF0A3EBF0900D8CE0FF900D9240
:107E7F00E0D39F4003027F5AA3128533128563908C
:107E8F000D94E0FEA3E0FFC39414EE9400502A90EB
:107E9F000D8E12855774272FF582E4340DF583ED7F
:107EAF00F0900D8FE004F07006900D8EE004F0124C
:107EBF0085BB70CB1285C280C6128530900D90F0B5
:107ECF00A3EFF0900D93128533128563900D8E12F0
:107EDF008599900D9012855412876D900D91E00445
:107EEF00F07006900D90E004F01285BB70031285C0
:107EFF00C2C3900D95E09414900D94E0940040CC83
:107F0F00128530900D90128566900D94E0FCA3E0E1
:107F1F00FDC39414EC94005022900D90128599AFEC
:107F2F00F0FE74272DF582E4340DF583E0FD128702
:107F3F006D1285BB70D31285C280CE128CF7900D57
:107F4F0092E004F0A3E004F0027E77900D12E0FFC0
:107F5F00900D8DE0FED39F5020900D8BE0FDA3E0A0
:107F6F00C39DFDE49400FCEE7A002DFDEA3CFCC3BA
:107F7F00ED9F7480F86C985013900D12E0FF900DE8
:0F7F8F008BE0D39F5009A3E0C39F4003128DA640
:017F9E0022C0
:0386E400900DB93D
:1086E70012858C128FEA900DBF1285A0900DBBF0FA
:1086F700900DB9E0FF900DBFE0FCA3E0FD7B017A90
:108707000D7927900DAF12854D128D64900DC0E045
:108717002414F0900DBFE03400F0900DBBE01285FB
:108727007FA374FFF0A3EAF0A3E9F0128FC8900DBE
:10873700BCA3E0FAA3E0AE02FF7A0D7927128548C1
:10874700128BEF128CF7900DBBE004F0E0C3941E80
:10875700409E128DA6900047E0FF128F7E900DBAC3
:05876700E024FF92AFC9
:01876C0022EA
:03885D00900DCFAC
:1088600012858C128FEA900DD21285A0900DD1F056
:10887000900DD1E0FFC3941E504175F014EF1285A6
:1088800037FE900DD4F0FAA3EFF0FB900DCFE0FF90
:10889000900DD2E0FCA3E0FDA9037BFF900DB71281
:1088A000854D128E56900DD3E02414F0900DD2E039
:1088B0003400F0900DD1E004F080B5900047E0FF67
:0B88C000128F7E900DD0E024FF92AFDD
:0188CB00228A
:03000000024000BB
:03000300025003A5
:03000B000250069A
:030013000250098F
:03001B0002500C84
:0300230002500F79
:03002B000250126E
:0300330002501563
:03003B0002501858
:0300430002501B4D
:03004B0002501E42
:0300530002502137
:03005B000250242C
:0300630002502721
:03006B0002502A16
:0300730002502D0B
:03007B0002503000
:03008300025033F5
:03008B00025036EA
:03009300025039DF
:03009B0002503CD4
:0300A30002503FC9
:10400000787FE4F6D8FD9000007F007E20E4F0A3E6
:0A401000DFFCDEFA75812102405545
:10401A00028989E493A3F8E493A34003F68001F2AA
:10402A0008DFF48029E493A3F85407240CC8C333A7
:10403A00C4540F4420C8834004F456800146F6DF76
:10404A00E4800B010204081020408090409AE47E2C
:10405A00019360BCA3FF543F30E509541FFEE4936B
:10406A00A360010ECF54C025E060A840B8E493A332
:10407A00FAE493A3F8E493A3C8C582C8CAC583CA5D
:10408A00F0A3C8C582C8CAC583CADFE9DEE780BE15
:01494C00006A
:10705B00E709F608DFFA8046E709F208DFFA803E17
:10706B0088828C83E709F0A3DFFA8032E309F60804
:10707B00DFFA8078E309F208DFFA807088828C836C
:10708B00E309F0A3DFFA806489828A83E0A3F60820
:10709B00DFFA805889828A83E0A3F208DFFA804CFA
:1070AB0080D280FA80C680D4806980F280338010D1
:1070BB0080A680EA809A80A880DA80E280CA80333A
:1070CB0089828A83ECFAE493A3C8C582C8CCC583B2
:1070DB00CCF0A3C8C582C8CCC583CCDFE9DEE78082
:1070EB000D89828A83E493A3F608DFF9ECFAA9F001
:1070FB00EDFB2289828A83ECFAE0A3C8C582C8CC57
:10710B00C583CCF0A3C8C582C8CCC583CCDFEADE6F
:10711B00E880DB89828A83E493A3F208DFF980CCD1
:10712B0088F0EF60010E4E60C388F0ED2402B404CA
:10713B000050B9F582EB2402B4040050AF23234571
:06714B0082239070AB737B
:10715100C2D530F707B2D563F0FF05F030E70CB2C6
:10716100D5F4048463F0FF05F080018430D502F486
:027171000422F6
:10717300BB010689828A83E0225002E722BBFE021A
:09718300E32289828A83E493224D
:10718C00BB010CE58229F582E5833AF583E02250B8
:10719C0006E92582F8E622BBFE06E92582F8E22202
:0D71AC00E58229F582E5833AF583E493221C
:1071B900BB010689828A83F0225002F722BBFE01B5
:0271C900F322AF
:1071CB00F8BB010DE58229F582E5833AF583E8F0FA
:1071DB00225006E92582C8F622BBFE05E92582C8A6
:0271EB00F2228E
:1071ED00C5F0F8A3E028F0C5F0F8E582158270022D
:0671FD001583E038F022CA
:10720300A3F8E0C5F025F0F0E5821582700215833E
:06721300E0C838F0E8229B
:10721900E88FF0A4CC8BF0A42CFCE98EF0A42CFC14
:107229008AF0EDA42CFCEA8EF0A4CDA8F08BF0A492
:107239002DCC3825F0FDE98FF0A42CCD35F0FCEBF1
:107249008EF0A4FEA9F0EB8FF0A4CFC5F02ECD39B6
:0F725900FEE43CFCEAA42DCE35F0FDE43CFC2223
:1072680075F008758200EF2FFFEE33FECD33CDCCDD
:1072780033CCC58233C5829BED9AEC99E582984060
:107288000CF582EE9BFEED9AFDEC99FC0FD5F0D63D
:10729800E4CEFBE4CDFAE4CCF9A88222B800C1B967
:1072A8000059BA002DEC8BF084CFCECDFCE5F0CBA5
:1072B800F97818EF2FFFEE33FEED33FDEC33FCEBDE
:1072C80033FB10D703994004EB99FB0FD8E5E4F999
:1072D800FA227818EF2FFFEE33FEED33FDEC33FC86
:1072E800C933C910D7059BE99A4007EC9BFCE99A7A
:1072F800F90FD8E0E4C9FAE4CCFB2275F010EF2FBF
:10730800FFEE33FEED33FDCC33CCC833C810D707BE
:107318009BEC9AE899400AED9BFDEC9AFCE899F8F9
:0E7328000FD5F0DAE4CDFBE4CCFAE4C8F9228C
:108B6900C2D5E830E70FB2D5E4C39BFBE49AFAE437
:108B790099F9E498F8EC30E717B2D5128B9F127285
:108B8900A4E4C39BFBE49AFAE499F9E498F8800316
:108B99001272A430D50DE4C39FFFE49EFEE49DFD4F
:048BA900E49CFC222A
:10733600EB9FF5F0EA9E42F0E99D42F0EC6480C8CE
:0673460064809845F0226E
:10734C00EB9FF5F0EA9E42F0E99D42F0E89C45F097
:01735C00220E
:0C735D00ECF0A3EDF0A3EEF0A3EFF022A3
:10736900A8828583F0D083D0821273801273801231
:107379007380127380E473E493A3C583C5F0C58356
:10738900C8C582C8F0A3C583C5F0C583C8C582C86E
:0173990022D1
:10739A00D083D082F8E4937012740193700DA3A382
:1073AA0093F8740193F5828883E473740293686096
:0673BA00EFA3A3A380DF96
:1073C000E50D2582F582E50C3583F583B50C048542
:1073D000820D2210AF0685820DF50C2285820DF5F7
:0473E0000CD2AF22FA
:0D73E400E50D2582F582E50C3583F5832249
:1073F100EC8EF0A4CCC5F0CCCDF8EFA4CEC5F02D29
:10740100FDE43CFCE8A42EC8C5F03DFDE43CFCEFE6
:0D741100A4FFE5F028FEE43DFDE43CFC2274
:10741E00EF4E6012EF60010EEDBB010B89828A8385
:10742E00F0A3DFFCDEFA2289F05007F709DFFCA992
:0C743E00F022BBFEFCF309DFFCA9F022E9
:00000001FF
